:100000000C94C2050C94DF050C94DF050C94DF05FD
:100010000C94DF050C94DF050C94DF050C94DF05D0
:100020000C94DF050C94DF050C941A270C94EC2734
:100030000C9463210C94DF050C94DF050C94DF0510
:100040000C94DF050C94DF050C94DF050C94DF05A0
:100050000C94DF050C94EB210C94DF050C94DF0568
:100060000C94DF050C94DF050C94DF050C94DF0580
:100070000C94DF050C94DF050C94DF050C94DF0570
:100080000C94DF050C94DF050C94DF050C94DF0560
:100090000C94DF050C94DF050C94DF050C94DF0550
:1000A0000C94DF050C94DF050C94DF05AD09AD0958
:1000B000D909D909410A5F0A770B770B6A0A030B42
:1000C000140B140B59288028782980287829CC28EB
:1000D000EF2878294629552929001E001F002000F5
:1000E00021002200230024002500260027002D00E7
:1000F0002E002A0049002B0014001A0008001500E9
:1001000017001C0018000C00120013002F00300014
:1001100031004C00354204001600070009000A00B7
:100120000B000D000E000F0033003400280000000B
:100130004B00E1001D001B00060019000500110026
:1001400010003600370038000000E50052004E0075
:10015000E000E300E200000000002C0000000000CE
:1001600000000151E600E400500051004F0035004E
:100170003A003B003C003D003E003F004000410093
:1001800042004300440045002A00A900010001008C
:100190000100520001000100010001000100010006
:1001A0000100010001000100AA000100010050004F
:1001B00051004F0001000100010001000100010099
:1001C0000100010000004A000100010001000100DF
:1001D000010001000100A800010001000100000071
:1001E0000100A8004D000100010001000000000016
:1001F0000100000000000000010001000100AC004F
:10020000AE00AB0035003A003B003C003D003E0034
:100210003F004000410042004300440045002A00E6
:10022000A9000100010001005200010001000100CD
:100230002400250026000100010001000100AA00A1
:1002400001000100500051004F0001000100210099
:100250002200230001000100010000004A0001000B
:100260000100010001000100010027001E001F0025
:100270002000010000000100A8004D000100010065
:10028000010000000000010000000000000001006B
:1002900001000100AC00AE00AB0044454255473AB6
:1002A0002064697361626C65642E0A00444542559E
:1002B000473A20656E61626C65642E0A000A00256B
:1002C000303258006C65645F7461736B3A20004F84
:1002D0006E6573686F743A206163746976653A205D
:1002E00025640A000A002530313662003A200025D4
:1002F000303258000A722F632030313233343536B1
:100300003738394142434445460A00290A002575D9
:10031000002F002575005D2800256400200025645D
:1003200000200025640020002564007C0025303278
:1003300058006D6F7573656B6579205B62746E7CB8
:10034000782079207620685D287265702F61636C53
:10035000293A205B00313A0964656C6179282A31B9
:10036000306D73293A2025750A323A09696E746531
:100370007276616C286D73293A2025750A333A0923
:100380006D61785F73706565643A2025750A343A4B
:100390000974696D655F746F5F6D61783A202575CA
:1003A0000A353A09776865656C5F6D61785F7370CF
:1003B0006565643A2025750A363A09776865656C83
:1003C0005F74696D655F746F5F6D61783A20257544
:1003D0000A00703A097072696E742076616C7565F6
:1003E000730A643A097365742064656661756C7498
:1003F000730A75703A092B310A646E3A092D310A75
:100400006C743A092B31300A72743A092D31300A72
:100410004553432F713A09717569740A0A737065FF
:100420006564203D2064656C7461202A206D6178CC
:100430005F7370656564202A202872657065617439
:10044000202F2074696D655F746F5F6D6178290A74
:1004500077686572652064656C74613A20637572B3
:10046000736F723D25642C20776865656C3D25644B
:100470000A53656520687474703A2F2F656E2E7765
:10048000696B6970656469612E6F72672F77696B3C
:10049000692F4D6F7573655F6B6579730A004D3E0B
:1004A00020004D25753A25733E20003F0A003D206F
:1004B00025750A003F0A0064656661756C74730AED
:1004C0000025750A003F0A000A092D2056616C7547
:1004D0006573202D0A00710A000A092D204D6F75E1
:1004E00073656B6579202D0A003F00433E20004C68
:1004F00025640A000A092D20537461747573202D38
:100500000A686F73745F6B6579626F6172645F6CA8
:1005100065647328293A20253032580A6B65796260
:100520006F6172645F70726F746F636F6C3A2025D5
:100530003032580A6B6579626F6172645F69646C0E
:10054000653A20253032580A74696D65725F7265AC
:100550006164333228293A202530386C580A000A61
:10056000092D2056657273696F6E202D0A56494415
:100570003A20307846454544284865787769726561
:1005800029205049443A20307836303630284D61A1
:10059000676963666F726365203638292056455255
:1005A0003A203078303030310A4255494C443A20B4
:1005B00020284665622032372032303232290A4FF5
:1005C0005054494F4E533A204C554641204D4F55BB
:1005D00053454B45592045585452414B45592043AA
:1005E0004F4E534F4C4520434F4D4D414E442034C8
:1005F0003039360A4743433A20352E342E302041D5
:1006000056522D4C4942433A20322E302E30204152
:1006100056525F415243483A20617672350A000AC9
:10062000092D20436F6E736F6C65202D0A4553436F
:100630002F713A09717569740A6D3A096D6F757396
:10064000656B65790A000A092D204D616769632091
:100650002D0A443A094465627567204D65737361DC
:10066000676520546F67676C650A583A094D617475
:10067000726978204465627567204D6F6465205407
:100680006F67676C65202D2053686F77206B6579E5
:100690007072657373657320696E206D6174726921
:1006A0007820677269640A4B3A094B6579626F6119
:1006B000726420446562756720546F67676C6520BB
:1006C0002D2053686F77206B657970726573732086
:1006D0007265706F72740A4D3A09446562756720DD
:1006E0004D6F75736520546F67676C650A563A09DC
:1006F00056657273696F6E0A533A09537461747563
:10070000730A433A09416374697661746520436FE3
:100710006E736F6C65204D6F64650A46312D4631EE
:10072000303A0953776974636820746F204C61799B
:10073000657220302D392028463130203D204C3044
:10074000290A302D393A0953776974636820746F28
:10075000204C6179657220302D390A475241564547
:100760003A0953776974636820746F204C61796526
:100770007220302028616C7465726E617465290A7C
:10078000423A094A756D7020746F20426F6F746C25
:100790006F616465720A4553433A094A756D70206A
:1007A000746F20426F6F746C6F6164657220286192
:1007B0006C7465726E617465290A453A09507269F4
:1007C0006E7420454550524F4D2053657474696EC8
:1007D00067730A4253504143453A09436C6561725D
:1007E00020454550524F4D0A006B65796D61705F31
:1007F000636F6E6669672E7261773A2025303258D2
:100800000A2E737761705F636F6E74726F6C5F63D3
:100810006170736C6F636B3A2025750A2E6361708B
:10082000736C6F636B5F746F5F636F6E74726F6C0A
:100830003A2025750A2E737761705F6C63746C5F64
:100840006C6775693A2025750A2E737761705F723F
:1008500063746C5F726775693A2025750A2E737729
:1008600061705F6C616C745F6C6775693A202575A7
:100870000A2E737761705F72616C745F726775695D
:100880003A2025750A2E6E6F5F6775693A202575C7
:100890000A2E737761705F67726176655F65736357
:1008A0003A2025750A2E737761705F6261636B73FE
:1008B0006C6173685F6261636B73706163653A203A
:1008C00025750A2E6E6B726F3A2025750A006465D5
:1008D0006275675F636F6E6669672E7261773A2033
:1008E000253032580A2E656E61626C653A20257596
:1008F0000A2E6D61747269783A2025750A2E6B652F
:1009000079626F6172643A2025750A2E6D6F757376
:10091000653A2025750A006565636F6E6669673AFA
:100920000A64656661756C745F6C617965723A2002
:1009300025750A003F000A6D6F7573653A206F6672
:10094000660A000A6D6F7573653A206F6E0A000AB9
:100950006B6579626F6172643A206F66660A000A9D
:100960006B6579626F6172643A206F6E0A000A6D7E
:1009700061747269783A206F66660A000A6D617464
:100980007269783A206F6E0A000A64656275673A88
:10099000206F66660A000A64656275673A206F6EAA
:1009A0000A000A0A4A756D70696E6720746F2062CA
:1009B0006F6F746C6F616465722E2E2E2000433E43
:1009C0002000436C656172696E6720454550524F47
:1009D0004D0A000A002530325820006B6579626F9D
:1009E0006172645F7265706F72743A20005B735D50
:1009F000005B575D005B535D005B525D005B445DD7
:100A0000005B435D001C034D0061006700690063EB
:100A10000066006F00720063006500200036003839
:100A2000000000100348006500780077006900723C
:100A300000650000000403090409025B00030100D3
:100A4000A0FA0904000001030101000921110100BD
:100A5000012240000705810308000109040100018B
:100A600003000000092111010001227B000705821B
:100A70000320000109040200020300000009211103
:100A8000010001222200070583032000010705035E
:100A9000032000011201000200000008EDFE60606A
:100AA0000100010200010631FF0974A10109751559
:100AB0000026FF009520750881020976150026FFA3
:100AC00000952075089102C005010902A101850267
:100AD0000901A1000509190129081500250195083A
:100AE000750181020501093009311581257F9502C3
:100AF0007508810609381581257F950175088106DD
:100B0000050C0A38021581257F950175088106C0FC
:100B1000C005010980A101850319012AB70015014B
:100B200026B700950175108100C0050C0901A101CF
:100B3000850419012AA002150126A002950175104D
:100B40008100C005010906A101050719E029E71583
:100B5000002501950875018102950175088101053F
:100B600007190029FF150026FF009506750881006A
:100B7000050819012905950575019102950175036F
:100B80009101C00011241FBECFEFDAE0DEBFCDBF60
:100B900011E0A0E0B1E0ECE6F4E502C005900D92B2
:100BA000AC3FB107D9F722E0ACEFB1E001C01D9234
:100BB000A23FB207E1F70E94BA170C94342A0C94B2
:100BC0000000FF93EF93E091FC01F091FD0130975D
:100BD00009F00995EF91FF910895FC01859180300E
:100BE00011F0EFDFFBCF0895FF27E0E230E247FF8F
:100BF0000CC0419597FF09C0EDE260957095809516
:100C00009095611D711D811D911D27FF02C02195C9
:100C100030E350E2AA27660F771F881F991FAA1F8B
:100C2000A41710F0A41B63955A95A9F7AA3008F0F1
:100C3000A95FA05DAF93F3956115710581059105DD
:100C400041F7ED3211F4EF93F395F21718F43F9357
:100C5000F395FBCF8F91B5DFFA95E1F70895E99110
:100C6000F9918591803021F0853219F0AADFF9CF12
:100C7000089520E0E89455915532C1F3503311F4B2
:100C8000689455915A3348F4505390F3220F022E32
:100C9000220F220F200D250FF4CF0EF421958991FC
:100CA0009991533619F3533729F1533559F1BC0152
:100CB00088279927E8945C3621F489919991689462
:100CC0005591543639F446EF7EF077FF0DC08FEF23
:100CD0009FEF0AC055374AE039F0583540E121F01E
:100CE000523642E009F00895FF93EF937DDFEF91D4
:100CF000FF91B7CFFF93EF93FC0181918030B9F35F
:100D000060DFFBCFFF93EF9368DFF1CFDF93CF93EB
:100D1000CDB7DEB72596A3DFCF91DF91089581E0AF
:100D2000089581E008950C94910608950C94950619
:100D30001F93CF93DF9300D000D01F92CDB7DEB7C3
:100D400049835A836B833091FF0189819A813111E4
:100D500014C0662359F0222349F00E94B40D182FC5
:100D6000682F89819A810E945D0D03C00E94880DC1
:100D7000182F69817A81812F04C00E94B40D698186
:100D80007A810F900F900F900F900F90DF91CF917D
:100D90001F910C94F814FC01262F4081518162812F
:100DA000738184810C94980681E00895CF93DF933A
:100DB000EC0160E00E94CB06BE01DF91CF910C9464
:100DC00096060C946B160C94671608950E94070CF7
:100DD0000E94E5062FEF84E39CE021508040904084
:100DE000E1F700C000000C9411220F931F93CF93E2
:100DF000DF938C0161E00E94CB06EC01B8010E94F8
:100E00009306882309F45BC0B801CE010E94F01F4D
:100E1000882309F454C0B801CE010E94D21A882355
:100E200009F44DC0B801CE010E944C1F882309F47B
:100E300046C0F80182818823D9F1CF3D8CE5D807DF
:100E400079F140F4C115FCE5DF0791F0C130DC45D4
:100E500091F02EC0CC35EDE5DE0741F1CD35FDE555
:100E6000DF0709F1CB35DD4519F50E944B1220C093
:100E70000E94E60624C080919802C82FC095C170D8
:100E8000C0FB80F980939802CC2329F08CEA92E091
:100E90000E94ED0514C08AE992E00E94ED0510C0A1
:100EA0000E94F9120CC00E94421202C00E944E120F
:100EB000C801DF91CF911F910F910C948F06C0E074
:100EC0008C2FDF91CF911F910F9108950E944521A2
:100ED0000C94A4070E94A7070C944B218295982F8D
:100EE000937344E0949F900111248C7C86958695A1
:100EF000282B822F8575880F2A7A2695822B0895B4
:100F0000CF93DF93D92F0E946E07C82F8D2F0E9499
:100F10006E072C2F30E0322F2227A901482BCA015F
:100F2000DF91CF91089508950C94930781E008957F
:100F30000C9496070895CF93C82F0E9494078C2F86
:100F40000E949807CF91089580E00C949B070E941F
:100F50004C200C949B07CF930E944C20C82F80916B
:100F6000FE01C81741F1C093FE018091980282FFF3
:100F70001EC080FF04C084EC92E00E94ED058091C9
:100F8000980280FF0CC01F92CF938FEB92E09F934B
:100F90008F930E9486060F900F900F900F90809174
:100FA000980280FF04C08DEB92E00E94ED058C2F2B
:100FB000CF910C949B07CF910895CF93DF93CDB73A
:100FC000DEB72B970FB6F894DEBF0FBECDBF4F83B1
:100FD000588769877A878B8761110E947A119E01F1
:100FE0002F5F3F4F86E0F90111928A95E9F785E07E
:100FF000FE013796D90101900D928A95E1F789811A
:101000009A814C815D81452B31F09F3F31F491E015
:101010008F3F19F403C091E001C090E090FF09C038
:1010200049815A816B817C818D819E810E949B10B8
:1010300005C0C9010E94D4068111F2CF2B960FB6CC
:10104000F894DEBF0FBECDBFDF91CF910895FC01B4
:10105000808191810E94F60D0895CF93882309F431
:10106000A9C0C82F8238C1F40E944C2081FDA2C0C3
:1010700069E380910201909103010E941D210E9469
:101080009C112FEF81EE94E0215080409040E1F7D9
:1010900000C0000069E319C0833801F50E944C20AC
:1010A00080FD88C063E580910201909103010E9458
:1010B0001D210E949C112FEF81EE94E02150804071
:1010C0009040E1F700C0000063E58091020190913B
:1010D00003010E941F21CF910C949C118438C1F40C
:1010E0000E944C2082FD66C067E4809102019091CD
:1010F00003010E941D210E949C112FEF81EE94E0BC
:10110000215080409040E1F700C0000067E4DDCF4F
:101110008CEF8C0F813AF8F48C2F0E94F51E811110
:1011200049C06C2F80910201909103010E94E72039
:10113000882349F06C2F80910201909103010E9455
:101140001F210E949C116C2F80910201909103013C
:101150000E941D21C0CF80E28C0F883048F4C770F8
:1011600081E001C0880FCA95EAF70E945D11B3CFF4
:10117000EBE5EC0FE33040F4F0E0E95BFE4F8081FB
:1011800090E0CF910C94AF20E8E5EC0FE73150F4FC
:10119000F0E0EE0FFF1FE75EFE4F80819181CF915F
:1011A0000C94C520CD3E30F08C2F0E943F18CF917B
:1011B0000C941119CF910895882309F464C08238E2
:1011C00079F40E944C2081FF5EC069E380910201A6
:1011D000909103010E941D210E949C1169E310C09F
:1011E0008338B1F40E944C2080FF4DC063E58091AC
:1011F0000201909103010E941D210E949C1163E550
:1012000080910201909103010E941F210C949C1176
:10121000843879F40E944C2082FF35C067E48091C5
:101220000201909103010E941D210E949C1167E41C
:10123000E7CF9CEF980F913A10F4682FE1CF90E23E
:10124000980F983050F4877091E001C0990F8A95FB
:10125000EAF7892F0E946311D9CF9BE5980F93304D
:1012600020F480E090E00C94AF2098E5980F97313F
:1012700020F480E090E00C94C5208D3E20F00E9488
:101280009A180C94111908951F93CF93DF93182F78
:10129000EB010E942D08209741F08FE99FE0019714
:1012A000F1F700C000002197F6CF812FDF91CF9199
:1012B0001F910C94DC08893319F060E070E002C0E3
:1012C00060E570E00C944409882321F00E945D11D0
:1012D0000C949C110895882321F00E9463110C94B2
:1012E0009C110895CF92DF92EF92FF920F931F937C
:1012F000CF93DF937C01D62FC72FFC01128105818C
:1013000002950F700E9453118823B9F01123A9F0A0
:101310008C2F807F803421F080E28D0F883068F040
:101320008091CC0282FD09C082E00E94FC110E94E3
:10133000531191E0D82ED92601C0D12CCC2EC294C5
:101340008FE0C8228C2D90E08C30910508F0CFC141
:10135000FC01EA5AFF4F0C94CB298C2F807FCF7071
:10136000882311F0C295C07F112399F0CC2309F492
:10137000AAC180E28D0F883010F0D11104C08C2FEB
:101380000E945D1103C08C2F0E946D110E949C1160
:101390009AC18D2F0E94DC08CC2309F4A8C180E2F9
:1013A0008D0F883038F1DD2329F18C2F0E947311C5
:1013B00024C08C2F807FCF70803211F0C295C07F07
:1013C000DD2319F0D130A1F13DC08091CC0282FF24
:1013D00017C0112349F0CC2329F08C2F0E945D11F6
:1013E0000E949C1180E070C180E00E94DC08CC2348
:1013F00009F47DC18C2F0E9463110E949C1177C15A
:10140000112371F0002341F0013031F40E947D116D
:101410008C2B0E9485116BC10E947D118C2B1DC0ED
:10142000002319F0013009F462C10E94921125C015
:10143000112321F0063008F05AC10EC0053008F023
:1014400056C11BC0112361F0002331F0F7018581E3
:1014500080FF39C18F7085838C2F0E94640947C13A
:10146000002359F0D93309F03FC1FFEF07EE13E035
:10147000F15000401040E1F735C18C2F0E946B09FC
:1014800036C18C2F86958695837019F0813061F076
:101490002EC1112321F08D2F9C2F937002C080E06C
:1014A00090E00E94AF202BC1112321F08D2F9C2FA3
:1014B000937002C080E090E00E94C52020C18D2F73
:1014C000112319F00E943F1802C00E949A180E942E
:1014D000111915C18C2F837009F047C011110BC170
:1014E0002D2F229526952770220F220F6D2F6F70BA
:1014F000862F90E0A0E0B0E0022E04C0880F991F74
:10150000AA1FBB1F0A94D2F7D4FF10C04FE050E0CF
:1015100060E070E004C0440F551F661F771F2A95D6
:10152000D2F7409550956095709503C040E050E02B
:10153000BA01C695C695C3708A019B01082B192B69
:101540002A2B3B2BC901B801C23049F058F4C130F5
:1015500019F00E94730CCFC00E94610CCCC00E9495
:10156000850CC9C00E945F0CC6C0112319F08C2FD6
:10157000817001C08695882309F4BDC02D2F229566
:1015800026952770220F220F6D2F6F70862F90E007
:10159000A0E0B0E0022E04C0880F991FAA1FBB1F55
:1015A0000A94D2F7D4FF10C04FE050E060E070E042
:1015B00004C0440F551F661F771F2A95D2F7409528
:1015C00050956095709503C040E050E0BA01C69513
:1015D000C695C3708A019B01082B192B2A2B3B2B24
:1015E000C901B801C23049F058F4C13019F00E9465
:1015F000380D81C00E94260D7EC00E944A0D7BC01E
:101600000E94990C78C0CF70112339F08C2F0E9462
:10161000BF0C8D2F0E9464096EC08D2F0E946B0934
:101620008C2F0E94E00C67C0D23F21F128F4D03FFC
:1016300041F0D13FC1F043C0D33F19F1D43F79F01D
:101640003EC0112341F0053008F051C08C2F8F713E
:101650000E94050D4CC0063008F049C0F7CF8091BC
:10166000CC0282FF18C0112339F08C2F8F710E9499
:10167000BF0C3DC01123C9F38C2F8F710E94E00C69
:1016800036C0112329F08C2F8F710E94AA0C2FC015
:101690000E94A50C2CC0112349F0CF718C2F0E9401
:1016A000BF0C63E08C2F0E94E11121C081E00E94F9
:1016B000FC110230E0F082E00E94FC1118C01123FE
:1016C00031F0002391F28D2F0E942D0810C00023CD
:1016D00099F2D93349F41FEF27EE33E0115020403F
:1016E0003040E1F700C000008D2F0E94DC0888EF39
:1016F0008C0D843020F40E944C200E949B07DD203A
:10170000C9F00E944F1180FD15C0F70112820E949E
:1017100049110E94BF0CC7010E94BB0B0E944911D6
:10172000DF91CF911F910F91FF90EF90DF90CF90BD
:101730000C94E00CDF91CF911F910F91FF90EF90EF
:10174000DF90CF9008950F931F93CF93DF93EC0119
:10175000688179818A810E94010E8C010E945C0D52
:101760000E944D0CB801CE010E947209DF91CF9109
:101770001F910F910895CF93DF93EC019881898198
:101780002B813C81232B31F08F3F31F481E09F3F4F
:1017900019F403C081E001C080E080FD1DC0CE01CE
:1017A0000E94F506811110C00E9453118823A1F0F8
:1017B0008A81882389F08091CC0282FD0DC082E06D
:1017C000DF91CF910C94FC11CE010E94A30BCE01AE
:1017D000DF91CF910C94D606DF91CF91089580E0F0
:1017E00090E00E94AF2080E090E00E94C5200E941F
:1017F0007A110E949C110E94C41A0C9411198091B4
:101800000201909103010E9421210C94EF0B0E9490
:101810006A110C94FF0B92959F70963079F010F43A
:10182000925001C09A50923068F4803F69F018F4E9
:10183000883E40F409C0843F29F406C0883E20F069
:10184000813F11F080E0089581E00895FC018081DE
:1018500091810E94F60D0E940B0C0895CF93DF93A7
:1018600000D000D01F92CDB7DEB70F900F900F9031
:101870000F900F90DF91CF910895CF93DF9300D019
:1018800000D000D0CDB7DEB726960FB6F894DEBFF5
:101890000FBECDBFDF91CF910895089508950C94A8
:1018A0004E0C0C944F0C0E94510C609336027093B6
:1018B000370280933802909339020C94EF0B0C940A
:1018C000530C0F931F930091360210913702209111
:1018D000380230913902602B712B822B932B1F9190
:1018E0000F910C94530C0F931F930091360210919B
:1018F000370220913802309139026023712382230C
:1019000093231F910F910C94530C0F931F930091ED
:101910003602109137022091380230913902602747
:101920007127822793271F910F910C94530C0C94CD
:101930004E0C0E94970C6093320270933302809396
:101940003402909335020C94EF0B60E070E0CB0111
:101950000C94990C0F931F9341E050E060E070E00D
:101960008A019B0104C0000F111F221F331F8A959B
:10197000D2F7C901B8011F910F910C94990C0F93E4
:101980001F9341E050E060E070E004C0440F551F39
:10199000661F771F8A95D2F78091320290913302A9
:1019A000A0913402B09135028A019B01082B192BBA
:1019B0002A2B3B2BC901B8011F910F910C94990C54
:1019C0000F931F9341E050E060E070E004C0440FCB
:1019D000551F661F771F8A95D2F7409550956095E1
:1019E00070958091320290913302A0913402B091AF
:1019F00035028A019B01082319232A233B23C901AD
:101A0000B8011F910F910C94990C0F931F9341E013
:101A100050E060E070E004C0440F551F661F771F60
:101A20008A95D2F78091320290913302A0913402CC
:101A3000B09135028A019B01082719272A273B27E5
:101A4000C901B8011F910F910C94990C0F931F932A
:101A5000009132021091330220913402309135020C
:101A6000602B712B822B932B1F910F910C94990C4F
:101A70000F931F9300913202109133022091340290
:101A80003091350260237123822393231F910F919C
:101A90000C94990C0F931F93009132021091330212
:101AA00020913402309135026027712782279327D5
:101AB0001F910F910C94990C08952FE0929F800D27
:101AC0001124E82FE695E695E695877051E001C070
:101AD000550F8A95EAF785E0E89FF0011124E05060
:101AE000FE4F20E030E070E04081CB01022E02C0CA
:101AF000969587950A94E2F78170819584278523CE
:101B0000842781932F5F3F4F2530310569F7089572
:101B10002FE0929F800D1124682F6695669566953B
:101B2000982F977085E0689FB001112440E050E045
:101B300080E0FB01E40FF51FE050FE4F208130E014
:101B4000092E02C0369527950A94E2F721703327B3
:101B5000042E01C0220F0A94EAF7822B4F5F5F4FD9
:101B60004530510531F70895BF92CF92DF92EF9241
:101B7000FF920F931F93CF93DF938C01C09032029B
:101B8000D0903302E0903402F0903502809136021A
:101B900090913702A0913802B0913902C82AD92A0F
:101BA000EA2AFB2ACFE1D0E0D701C6010C2E04C0FF
:101BB000B695A795979587950A94D2F780FD04C0AE
:101BC000219790F7B12C07C0BC2EB8018C2F0E9432
:101BD0000B150197A9F38B2DDF91CF911F910F91D9
:101BE000FF90EF90DF90CF90BF900895CF93DF9359
:101BF000EC010E94B40DBE010E940B15DF91CF9144
:101C000008951F93CF93DF93EB019091FF019923E8
:101C100021F0CB010E94F60D13C0882349F0CB01BF
:101C20000E94B40D182F682FCE010E945D0D04C0D4
:101C3000CB010E94880D182FBE01812F0E940B1529
:101C4000DF91CF911F9108951F93CF93DF93C091A0
:101C50003A0216E080913B02C81799F0D0E01C9F31
:101C6000F0011D9FF00D1124E45CFD4F4081518176
:101C700062817381848195810E943D0C2196C77099
:101C8000E9CFDF91CF911F91089540916C0250915F
:101C90006D0260916E0270916F028091700290915E
:101CA00071020C943D0CEF92FF920F931F93CF9310
:101CB000DF938091710282958F7009F065C08091E9
:101CC0006E02882309F460C080913A02F0903B02D2
:101CD00010916C0200916D0260916F027091700220
:101CE00091E01F3F09F090E0C0910001D091010107
:101CF000292F96E0E92E8F1509F446C0611571056C
:101D000021F00F3F21F030E003C031E001C0322F5D
:101D100090E030FD36C0E89EF001E99EF00D112400
:101D2000DF01A45CBD4F11963C911197301329C07F
:101D30003C91311326C012963C911297311121C06B
:101D400013964D915C911497461B570B4C175D07EA
:101D5000C0F4809171028F70806180937102EF5B9B
:101D6000FD4F80818F70806180838CE692E00E94BD
:101D7000BB0BDF91CF911F910F91FF90EF900C94CF
:101D8000240E01968770B7CFDF91CF911F910F91ED
:101D9000FF90EF9008959F92AF92BF92CF92DF9203
:101DA000EF92FF920F931F93CF93DF93CDB7DEB7E0
:101DB00061970FB6F894DEBF0FBECDBF8C0185E0F2
:101DC000F801DE011D9601900D928A95E1F7D80188
:101DD0001296EC9090916C02E0916D0220916F024E
:101DE000309170022115310531F0EF3F31F481E07F
:101DF0009F3F19F403C081E001C080E0B82FB170AB
:101E00009B2E80FD47C1D8014C9111965C91119792
:101E10001396AD90BC9014978CE6C82E82E0D82E15
:101E2000F0906E02B501621B730B2091000130919E
:101E30000101FF2009F4D9C0809171026217730774
:101E400008F095C0282F207F09F052C05E1313C000
:101E5000491311C0FE2CE1100EC08F708061809379
:101E600071020E94450EC6010E94BB0B8091710257
:101E7000F80185834DC1AB2831F05F3F31F481E03B
:101E80004F3F19F403C081E001C080E080FD03C032
:101E900081E08E2502C080E090E0F82FF170FF2EE7
:101EA00080FF1CC080913A0220913B0236E08217ED
:101EB00009F40BC190E0389FF001399FF00D112417
:101EC000E45CFD4F6181561306C06081461303C078
:101ED0006281E61203C001968770E9CFFE2CEE20E6
:101EE00009F416C18091710281608093710254C01F
:101EF0005E1306C0491304C0E11002C0F80199C086
:101F0000C8010E94260C882361F1EE2051F1209136
:101F10007102822F82958F7090E0029774F0809109
:101F20006C0290916D0298878F831986BB86AA8672
:101F30002C87CE0107960E94BB0B86E0F801ACE629
:101F4000B2E001900D928A95E1F70E94530E0E9433
:101F5000450E0AC05E1711F1C8010E94260C8111BE
:101F60002CC0C8010E94BB0BFF24F394D1C0282FC2
:101F7000207F81F77A2DB98AA88A6E2D89890E94DF
:101F80002E0C8CE692E00E94BB0B86E0D6011D92DF
:101F90008A95E9F70E94450EF12CBAC04913DCCFAF
:101FA000E110DACFF8018583C8010E94BB0B86E0FF
:101FB000D6011D928A95E9F7ABC0EE2091F22091EF
:101FC0007102822F82958F7090E002970CF4B5CF4A
:101FD00080916C0290916D029A8389831B82BD82ED
:101FE000AC822E83CE010196A6CF6217730708F04C
:101FF00044C0FE2CEE2009F4B4CF5E1330C0491368
:102000002EC02091710220FD21C0822F82958F70F9
:10201000482F50E041155105C9F0F80125834F3094
:10202000510541F08F5F982F9295907F822F8F708E
:10203000892B8583C8010E94BB0B86E0F801ACE6C2
:10204000B2E001900D928A95E1F73CC086E0F8017C
:10205000ACE6B2E001900D928A95E1F759C0C80153
:102060000E94260C811169CF80917102816080935A
:102070007102C8010E94BB0B4BC07A2DB98AA88A95
:102080006E2D89890E942E0C86E0D6011D928A95BC
:10209000E9F718C0EE2009F464CFC8010E94260CAD
:1020A000F82E882309F45DCF86E0F801ACE6B2E0B3
:1020B00001900D928A95E1F78CE692E00E94270844
:1020C0000E94530E0E94450E23C04D875E878D856A
:1020D0009E850E94F60D292F22952F70223028F41C
:1020E0009F7039F0811105C00BC0243028F49F7017
:1020F00049F4805E883020F0C8010E94BB0B9F2C01
:10210000F92C06C0D80115969C91907F91F7F8CFD5
:102110008F2D61960FB6F894DEBF0FBECDBFDF9155
:10212000CF911F910F91FF90EF90DF90CF90BF90D4
:10213000AF909F9008951F93CF93DF93CDB7DEB7F5
:102140002C970FB6F894DEBF0FBECDBF4F835887D4
:1021500069877A878B879C87CE0107960E94CB0E72
:102160008823D1F09F8188852A853B85232B31F0F8
:102170008F3F31F481E09F3F19F403C081E001C03B
:1021800080E080FD47C04F81588569857A858B85C1
:102190009C850E943D0C3EC086E0FE013796DE0124
:1021A000119601900D928A95E1F7FF81E8856A8585
:1021B0007B856115710531F0EF3F31F481E0FF3F20
:1021C00019F403C081E001C080E080FD23C02091AC
:1021D0003B0230E0C90101968770992740913A028D
:1021E00050E084179507F1F1F983EA837D836C83CE
:1021F00096E0929FD001939FB00D1124A45CBD4F37
:10220000FE01319601900D929A95E1F780933B0281
:102210000E94240E16E080913A0290913B028917A9
:1022200071F1189FC0011124845C9D4F0E94CB0E58
:10223000882329F1E0913A021E9FF0011124E45C09
:10224000FD4F4081518162817381848195810E941B
:102250003D0C80913A0290E0019687709927809317
:102260003A02D9CF0E94070C10923B0210923A0218
:10227000ECE6F2E086E0DF011D928A95E9F72C9604
:102280000FB6F894DEBF0FBECDBFDF91CF911F9187
:10229000089580917A028595859585950895809118
:1022A0007A028770089590917A02977081E009F41C
:1022B00080E0089580918502089590918502892B90
:1022C000809385020895809590918502892380935B
:1022D0008502089510928502089590918402892BB9
:1022E000809384020895809590918402892380933D
:1022F0008402089510928402089580917B020895CB
:1023000008950C9480110C9481119091CC0292FD4F
:1023100008C090917B02981721F080937B020C9467
:102320008311089580917B02882329F010927B020B
:1023300080E00C9483110895CF93DF93E091020124
:10234000F0910301809185028083E0910201F09178
:102350000301908180918402892B808380917B028C
:10236000882381F0E0910201F09103019081892B93
:10237000808380910201909103010E94DB208111F2
:102380000E949211C0910201D091030148E050E0F7
:1023900062E772E0CE010E94E529892B69F088E0AE
:1023A000FE01A2E7B2E001900D928A95E1F7CE011D
:1023B000DF91CF910C945820DF91CF9108950C9428
:1023C00080119091CC0292FD10C098E0899F9001FD
:1023D0001124262B20937A020E94BF0C80917A024E
:1023E0008595859585950C94DF110C94BF0C109202
:1023F0007A0280E00C94DF1120917A02809582238A
:1024000080937A02982F977099F430E0482F082E25
:10241000000C550B2417350759F09091CC0292FD12
:1024200007C08595859585950E94E00C0C94F71161
:102430000895CF939091CC0292FB222720F9281780
:10244000F9F0C82F892FC0FB82F98093CC028091CC
:10245000CB029091CC020E94751282E00E94FC1186
:102460008091980280FF0CC01F92CF938FEC92E076
:102470009F938F930E9486060F900F900F900F905E
:10248000CF9108958091CC0282FB882780F991E05A
:1024900089270C94191281E00C94191280E00C9495
:1024A000191280E090E00E94FA2921E0893E9E4FB7
:1024B00009F020E0822F089582E090E00C94F22948
:1024C00083E090E00C94F229CF9384E090E00E94A6
:1024D000F229C82F82E290E00E94F2292C2F30E0EE
:1024E000A901582BCA01CF910895CF93C92F682F06
:1024F00084E090E00E94002A6C2F82E290E0CF916D
:102500000C94002AAB01BC018FE090E00C94122ADD
:10251000AB01BC0183E190E00C94122A60E070E012
:10252000CB010C94881260E070E0CB010E94821213
:102530000C948E1269EE7EEF80E090E00E941E2ADD
:1025400060E082E090E00E94002A60E083E090E09A
:102550000E94002A1092360210923702109238021E
:102560001092390260E084E090E00E94002A60E06E
:1025700082E290E00E94002A60E085E090E00E9404
:10258000002A60E086E090E00E94002A6FEF87E07A
:1025900090E00E94002A40E050E0BA0188E090E01C
:1025A0000E94122A60E08DE090E00E94002A40E044
:1025B00050E0BA0188E190E00E94122A60E087E1D1
:1025C00090E00E94002A40E050E0BA018CE190E0E7
:1025D0000E94122A60E070E080E290E00E941E2AD1
:1025E00040E050E0BA0188E190E00E94122A0C9489
:1025F00093120C949A12682F8EE090E00C94002AAB
:102600000E94D02160939402709395028093960269
:10261000909397026093900270939102809392023C
:1026200090939302089585B7806885BF85B78068C9
:1026300085BF089581E008950C941A1308950C94B1
:102640001E130C941E130C9421130C941E130C9443
:1026500025130C941E130E94131385EF93E20E941E
:1026600042200E9429130C9427130E941F130C94DC
:102670001E130E94E8150C949A070E94BB210E9429
:1026800013170E9439130C9423135F926F927F9259
:102690008F929F92AF92BF92CF92DF92EF92FF9272
:1026A0000F931F93CF93DF93CDB7DEB72A970FB663
:1026B000F894DEBF0FBECDBF0E942817C82E81112F
:1026C0000E94001336E8832E32E0932E00E010E0E3
:1026D000502E802F0E940C165C01F40161907190C5
:1026E0004F016826792661147104B1F40F5F1F4F02
:1026F0000530110569F78FEF89838A831B820E9459
:10270000C4218160782F9D838C8349815A816B819C
:102710008D810E94DD073AC08091980281FD0E9460
:102720001516D12CEE24E394F12CC3018E219F21A8
:10273000892B29F10E941C138823A9F0DE825F8275
:10274000AE20BF2081E0AB2809F480E088870E949A
:10275000C4218160782F9A8789874E815F8168853F
:102760008A850E94DD07000F111FF801EA57FD4F0F
:1027700080819181E826F926F182E08207C0D39416
:10278000EE0CFF1CFFE0DF12D0CFB0CF81E0C11014
:1027900001C080E02A960FB6F894DEBF0FBECDBF11
:1027A000DF91CF911F910F91FF90EF90DF90CF902D
:1027B000BF90AF909F908F907F906F905F900895A3
:1027C0000E9445130E94B1190C94AB07CF93DF937D
:1027D0000E941015EC01811521E5920708F045C013
:1027E000811530E5930708F094C0883E910528F5DF
:1027F000803E910508F0F8C0883A910570F4853A5A
:10280000910508F07CC08130910509F475C008F489
:10281000E8C0049708F0E8C0E4C08F3B910508F0D9
:10282000E0C0C85AD0E0CC0FDD1FC65BDE4F099078
:10283000D881C02DCE019464D8C0811540E29407A0
:1028400058F4811551E0950708F0CEC08D3E9105F2
:1028500008F4C7C09065C9C0C11580E4D80708F462
:10286000C0C0DF70CE01906AC0C0811525E5920717
:10287000A8F4811534E5930708F095C0811543E568
:10288000940708F07BC0811552E5950708F061C0F8
:10289000D82FCC27CE01816F906AA7C0C11589E5DA
:1028A000D807A0F4C11528E5D20708F082C0C115E9
:1028B00036E5D30708F095C08C2F0E94A4158F71C0
:1028C00090E0D82FCC27CE0190628FC0C1154AE589
:1028D000D40708F474C0CE0190568115904208F0D8
:1028E00080C08D2F8F710E94A415DD27D0628F715B
:1028F000AE01582BCA0179C081E090E076C0C55A7C
:10290000D0E0C858DE4F8881C82FD0E0CE01906457
:102910006CC074E0969587957A95E1F7282F23701F
:102920003C2F337081E090E002C0880F991F3A95E8
:10293000E2F79C68AC01522B9A019C2F9F709695F0
:10294000969550E2959FE0011124C9018C2B9D2B97
:102950004CC08370992721E030E002C0220F331F62
:102960008A95E2F79C2F9695969580E2989FE001D4
:102970001124C22BD32BCE019C6837C083709927BA
:1029800021E030E002C0220F331F8A95E2F79C2F2E
:102990009695969540E2949FE0011124C22BD32B8B
:1029A000CE019A6822C0D82FCC27CE01846F906ABE
:1029B0001CC0DC2FCC27CE01806F906A16C08C2FF4
:1029C0008F700E94A41594E0D695C7959A95E1F76B
:1029D000CF70D0E0DC2FCC27D0699E01282BC90115
:1029E00004C080E090E001C0CE01DF91CF91089556
:1029F0002BE4829FC0011124FC012FE0729FE00DA7
:102A0000F11D1124E60FF11DEE0FFF1FE852FF4FDD
:102A10008591949108950E94F8140E94E6130895F8
:102A20008238910569F1B0F48133910509F46DC0E4
:102A300048F48932910509F463C08A32910509F49A
:102A400069C008958533910509F455C0893391050E
:102A5000B9F00895833E910569F138F4803E9105FF
:102A6000B1F0823E910509F10895863E9105A9F1E4
:102A7000873E9105B9F1843E910509F064C023C0F9
:102A80002091CB0220FD4FC021FD4DC008958091C3
:102A9000CB0280FD44C08091CC0280FF44C0809175
:102AA000CB0284FD42C083EE4DC08091CB0282FFF9
:102AB00038C0F5CF8091CB0282FD33C08091CC022B
:102AC00080FD31C0ECCF8091CC0281FF32C080917B
:102AD000CB0284FD2AC087EE35C08091CB0283FFF4
:102AE00026C0F5CF8091CB0283FD21C08091CC021E
:102AF00081FD1FC0ECCF8091CB0285FD1CC01DC0A5
:102B00008091CB0285FD19C016C08091CB0286FD55
:102B100016C017C08091CB0286FD13C010C089E398
:102B200011C082EE0FC080EE0DC080E00BC086EEBB
:102B300009C084EE07C089E205C085E303C08AE2CC
:102B400001C081E390E008959091CB0292FF0DC007
:102B5000282F2871283019F4877F846006C0282F19
:102B60002471243011F48B7F886093FF0DC0282FCF
:102B70002871283119F4877E846106C0282F2471BA
:102B8000243111F48B7E88612091CC0220FF0DC08E
:102B9000382F3871383019F4877F816006C0382F9C
:102BA0003171313011F48E7F886021FF0DC0282FE4
:102BB0002871283119F4877E816106C0282F217180
:102BC000213111F48E7E886194FD877E08950895E9
:102BD0000E945112811102C00E94F9120E945C12DF
:102BE000809398020E9464129093CC028093CB024F
:102BF0000E94E7150E946012682F70E080E090E06C
:102C00000E945F0C60913202709133028091340215
:102C1000909135020C94970CE82FF0E0EE0FFF1F17
:102C2000E952FD4F808191810895CF92DF92EF921A
:102C3000FF920F931F93CF93DF9384EF92E00E9454
:102C4000ED0587EDE82E82E0F82EC0E0D0E09FEEA3
:102C5000C92E92E0D92E06EE12E0DF93CF93DF92D9
:102C6000CF920E9486068CEE92E00E94ED05F7015D
:102C7000819191917F010E9480079F938F931F9371
:102C80000F930E94860684EE92E00E94ED05219645
:102C90008DB79EB708960FB6F8949EBF0FBE8DBF36
:102CA000C530D105D1F6DF91CF911F910F91FF90E3
:102CB000EF90DF90CF90089580EA8A95F1F708951C
:102CC00000C008950C945C1608950C9464160C943E
:102CD00065160C9464160C946916F894E82FE29526
:102CE000EF70F0E031A1282F2F7081E090E001C05B
:102CF000880F2A95EAF7982F9095932391A392A194
:102D0000892B82A3789408950F931F93CF93DF9319
:102D1000CAE8D1E089918F3F11F00E946D1681E0E1
:102D2000CF38D807B9F7CBE7D1E00AE811E08991AD
:102D30008F3F11F00E946D160C171D07C1F7DF9130
:102D4000CF911F910F910895BF92CF92DF92EF9292
:102D5000FF920F931F93CF93DF938C01C62FD0E088
:102D6000CE0186579E4F6C01FC0190819F3F09F474
:102D700050C0B62EF894E92FE295EF70F0E081A1F3
:102D80009F7021E030E001C0220F9A95EAF7822B74
:102D900081A382A12095282322A378940E94601603
:102DA000EBE7F1E04AE851E021E030E0E12CF12CE2
:102DB00061916F3F89F0A62FA295AF70B0E0909619
:102DC0008C9190E06F7002C0959587956A95E2F7B7
:102DD00080FD02C0C90102C080E090E0E82AF92A23
:102DE000220F331F4E175F0719F7F60180818F3FBF
:102DF00011F00E946D1661E0E114F10409F460E045
:102E00008B2D0E946216CC0FDD1FC00FD11FF982DF
:102E1000E882DF91CF911F910F91FF90EF90DF90AB
:102E2000CF90BF9008950E9484168AE0E7EDF2E00B
:102E3000DF01982F1D929A95E9F7EDECF2E0DF01A2
:102E40001D928A95E9F785E00E9473170C94E106BC
:102E5000FF920F931F93CF93DF93CDB7DEB72A97DF
:102E60000FB6F894DEBF0FBECDBF8E010F5F1F4FB0
:102E70008AE0F80111928A95E9F7F12C6F2DC801CB
:102E80000E94A416F394F5E0FF12F8CF4AE050E058
:102E9000B8018DEC92E00E94E529FF24F39400979D
:102EA00009F4F12C892B41F08AE0F801ADECB2E095
:102EB00001900D928A95E1F72F2D45E067ED72E0C4
:102EC0008DEC92E00E9474170E94E3068F2D2A96E3
:102ED0000FB6F894DEBF0FBECDBFDF91CF911F912B
:102EE0000F91FF9008950895FF920F931F93CF9332
:102EF000DF93F82E092F162FD72FC42F222349F046
:102F000081E080939B020E94C42190939A02809357
:102F1000990280919B028823D9F080919902909127
:102F20009A020E94DC21059798F0EF2DF02FA12F37
:102F3000BD2F80E090E04C2F50E08417950734F4CB
:102F4000219131912D933D930196F7CF10929B02E1
:102F5000DF91CF911F910F91FF9008950E947124EE
:102F60000E943D130C947D240E9481240E94E01352
:102F70000C949F240E9462210E9458240E942B13CB
:102F80000E94AE170E94B4170E943513FBCF8091A8
:102F9000A20280FF06C06091090170E0660F771FF2
:102FA00026C081FF04C06091090184E005C082FF52
:102FB00007C06091090188E0689FB001112417C023
:102FC0009091A1029923D1F060910801961788F79A
:102FD0002091090188E0289F90011124929FA0016F
:102FE000939F500D112470E0CA010E94B7296038E8
:102FF000710540F46115710519F406C068E070E0D0
:10300000862F08958FE7089581E008958091A202A8
:1030100080FF08C06091050170E075956795759512
:10302000679521C081FF06C06091050170E075952C
:10303000679519C082FF04C06091050170E010C05F
:103040009091A002992399F0609104019617A0F73E
:1030500080910501899FC001112470E00E94B72969
:103060006038710540F46115710519F406C061E01E
:1030700070E0862F08958FE7089581E008958D3ED2
:1030800021F40E94C717819504C08E3E29F40E9446
:10309000C7178093A60208958F3E21F40E94C71798
:1030A000819504C0803F29F40E94C7178093A50230
:1030B0000895893F19F40E94061805C08A3F31F42B
:1030C0000E94061881958093A70208958B3F21F4F2
:1030D0000E940618819504C08C3F29F40E940618AE
:1030E0008093A80208959FE0980F983078F421E02B
:1030F00030E0A90102C0440F551F9A95E2F7CA01BA
:103100009091A402892B8093A40208958D3F21F40D
:103110008091A20281600BC08E3F21F48091A202B7
:10312000826005C08F3F29F48091A2028460809361
:10313000A20208958D3E39F49091A60297FF35C002
:103140001092A60259C08E3E29F49091A60219163B
:10315000BCF32BC09091A5028F3E29F497FF25C0A8
:103160001092A50249C0803F19F41916CCF31DC076
:103170009091A702893F29F41916BCF41092A70276
:103180003BC08A3F19F497FF10C0F8CF8B3F39F44A
:103190009091A80297FF09C01092A8022DC08C3F01
:1031A00021F49091A8021916BCF39FE0980F983073
:1031B00080F421E030E0A90102C0440F551F9A9528
:1031C000E2F7CA0180959091A40289238093A4021A
:1031D00013C08D3F21F48091A2028E7F0BC08E3FE1
:1031E00021F48091A2028D7F05C08F3F29F4809148
:1031F000A2028B7F8093A2028091A502811106C05A
:103200008091A602811102C01092A1028091A702B2
:10321000811106C08091A802811102C01092A00203
:1032200008958091980283FF7EC082E393E00E941C
:10323000ED058091A4021F928F938DE293E09F93FE
:103240008F930E9486068BE293E00E94ED058091A9
:10325000A502282F082E000C330B3F938F9388E292
:1032600093E09F938F930E94860686E293E00E94EC
:10327000ED058091A602282F082E000C330B3F93FA
:103280008F9383E293E09F938F930E94860681E25F
:1032900093E00E94ED058091A702282F082E000CD4
:1032A000330B3F938F938EE193E09F938F930E9414
:1032B00086068CE193E00E94ED058091A802282FFC
:1032C000082E000C330B3F938F9389E193E09F937B
:1032D0008F930E94860686E193E00E94ED0580911F
:1032E000A1021F928F9383E193E09F938F930E949B
:1032F000860681E193E00E94ED058091A2021F9273
:103300008F938EE093E09F938F930E9486068BE0CD
:1033100093E00E94ED058DB79EB74C960FB6F894DA
:103320009EBF0FBE8DBF0E94C4212091A502211116
:1033300004C02091A602222321F090939F02809343
:103340009E022091A702211104C02091A8022223ED
:1033500021F090939D0280939C0283EA92E00C946A
:10336000A120EF92FF920F931F93CF93DF9300D092
:1033700000D000D0CDB7DEB786E0E3EAF2E0DE01B0
:10338000119601900D928A95E1F7E090A502F090D8
:10339000A6020091A7021091A8021092A502109215
:1033A000A6021092A7021092A802E11003C0FF200B
:1033B00009F45DC080919E0290919F020E94DC21E1
:1033C000AC019091A102992339F020910A0130E0DB
:1033D0002417350758F04BC020910B018AE0289F35
:1033E000900111242417350718F041C09F3F19F0B0
:1033F0009F5F9093A102EE2061F00E94C7171E14F8
:1034000014F09FEF01C091E0989F902D11249093AC
:10341000A502FF2061F00E94C7171F1414F09FEF50
:1034200001C091E0989F902D11249093A6023091B5
:10343000A5023323E1F02091A6022223C1F045EB3F
:103440003403C0011124992319F09093A50203C0FD
:1034500081E08093A50235EB2303C0011124992359
:1034600019F09093A60203C081E08093A602011197
:1034700003C0112309F45DC080919C0290919D02CC
:103480000E94DC21AC019091A002992339F0209197
:10349000060130E02417350758F04BC02091070192
:1034A0008AE0289F900111242417350718F041C0A5
:1034B0009F3F19F09F5F9093A002002361F00E944C
:1034C0000618101614F09FEF01C091E0989F902D00
:1034D00011249093A702112361F00E94061811167F
:1034E00014F09FEF01C091E0989F902D11249093CC
:1034F000A8023091A7023323E1F02091A8022223F1
:10350000C1F045EB3403C0011124992319F09093C5
:10351000A70203C081E08093A70235EB2303C0011B
:103520001124992319F09093A80203C081E080939D
:10353000A8028091A50281110BC08091A602811181
:1035400007C08091A702811103C08091A802811158
:103550000E941119EB82FC820D831E8386E0FE011E
:103560003196A3EAB2E001900D928A95E1F7269692
:103570000FB6F894DEBF0FBECDBFDF91CF911F9184
:103580000F91FF90EF900895E3EAF2E086E0DF010B
:103590001D928A95E9F71092A1021092A002109252
:1035A000A2020895CF93DF93EC01FB01828188236F
:1035B00009F43CC1C430FDE5DF0760F4CB3F9CE576
:1035C000D90788F49E0122503C452431310508F08A
:1035D0002EC109C0C236EDE5DE0729F0C63AFDE589
:1035E000DF0709F024C10E9464129093CC028093FB
:1035F000CB02C1318CE5D80709F4C6C008F042C03F
:10360000C930ECE5DE0709F49BC000F5C5308CE558
:10361000D80709F485C078F4C330ECE5DE0709F477
:1036200078C008F07AC0C230DC4509F0F5C080915E
:10363000CB028160EFC0C7309CE5D90709F478C0A0
:1036400008F07AC08091CB028061E4C0CD30FCE507
:10365000DF0709F487C058F4CB309CE5D90709F49B
:1036600079C008F07BC08091CB0288606FC0CF30FA
:10367000FCE5DF0709F480C008F082C08091CB022E
:10368000877FC8C0CE3F9CE5D90709F471C000F51B
:10369000C531FCE5DF0709F485C068F4C3319CE55A
:1036A000D90709F475C008F095C00E94070C8091F5
:1036B000CB028F77AFC0CC3FFCE5DF07A9F108F064
:1036C00054C0CB3FDC4509F0A7C08091CC0240C07C
:1036D000C230EDE5DE0709F489C058F4C1158DE567
:1036E000D80709F45AC008F069C08091CC02826002
:1036F0002FC0C236EDE5DE0709F47CC0C63AFDE511
:10370000DF0709F481C0C330DD4509F085C080E0E2
:103710006EC08091CB0282607DC08091CB0216C0CA
:103720008091CB02886076C08091CC0282604FC0CD
:103730008091CB0280626EC08091CB0280646AC0AF
:103740000E94070C8091CB02806864C0846062C0D4
:1037500081603DC08091CB028E7F5CC08091CB02A6
:103760008D7F58C08091CB0216C08091CC0218C0CA
:103770008091CC028D7F2BC08091CB028F7E4AC07E
:103780008091CB028F7D46C08091CB028F7B42C05F
:103790008091CB02877F8B7F3DC08091CC028D7F53
:1037A0008E7F15C08091CB0282FB222720F991E009
:1037B000922790FB82F990FB83F92CC08091CC0278
:1037C000982F909591708E7F892B90FB81F9809333
:1037D000CC0222C00E94070C8091CB0287FB2227DB
:1037E00020F991E0922790FB87F914C081E00E94B4
:1037F000FB1212C08091CB0284FB222720F991E0BA
:10380000922790FB84F906C08091CB02982F909567
:1038100090FB80F98093CB028091CB029091CC02F7
:103820000E9475120E94070C80E001C081E0DF91C8
:10383000CF910895809104011F928F93809105018B
:103840001F928F93809108011F928F93809109019D
:103850001F928F9380910A011F928F9380910B0189
:103860001F928F9385E593E09F938F930E94860626
:103870008DB79EB70E960FB6F8949EBF0FBE8DBF44
:103880000895883220F58E3108F068C08B3091F1B0
:10389000C0F4873009F0BEC081E080930B0184E161
:1038A00080930A018AE0809309018EE180930801E8
:1038B00088E08093050188E28093040187EB94E01F
:1038C000C6C0833109F443C0843169F1A3C08F3489
:1038D00009F49EC028F4893231F1883359F09AC036
:1038E000813531F008F4D4C0823509F4A7C092C004
:1038F0008FEFA5C089ED94E00E94ED050E941A1C8F
:103900001F9281E08F931F9288E08F9382ED93E066
:103910009F938F930E9486060F900F900F900F90A9
:103920000F900F9096C086ED94E00E94ED05809177
:10393000AD02882309F4AAC01092AD021092AC0225
:103940001092AB021092AA021092A902B1C088ECA8
:1039500094E00E94ED050E941A1C7BC08D5180935B
:10396000AD02833031F170F48130D1F0823009F052
:103970003FC08AE091E09093AC028093AB028CE967
:1039800091E01FC0853059F108F1863089F584E057
:1039900091E09093AC028093AB0287ED91E011C06F
:1039A0008BE091E09093AC028093AB0283E991E0CD
:1039B00008C089E091E09093AC028093AB0288EA62
:1039C00091E09093AA028093A90218C088E091E048
:1039D0009093AC028093AB0285EB91E0F2CF85E04F
:1039E00091E09093AC028093AB0284EC91E0E9CF3C
:1039F0001092AD0285EC94E00E94ED058091AD023D
:103A0000882309F455C01F928F9381EC94E00DC078
:103A10008AE015C084EB94E01AC097FF47C010827B
:103A200080811F928F938EEA94E09F938F930E94E0
:103A300086060F900F900F900F900BC081E0E091E1
:103A4000AB02F091AC02309729F58BEA94E00E942A
:103A5000ED052091AD02222359F18091A9029091A8
:103A6000AA02009711F48FE891E09F938F931F9221
:103A70002F9382EA94E09F938F930E9486060F9083
:103A80000F900F900F900F900F9016C080E0089548
:103A900086EFD5CF2081082E000C990B820F911D47
:103AA0008F3F910509F00CF4B8CF8FEF8083B8CF2A
:103AB0008EE994E00E94ED0581E00895CF93C82F30
:103AC0001F928F938FEE94E09F938F930E948606B0
:103AD00081E090E0A0E0B0E0BC01CD0104C0660F41
:103AE000771F881F991FCA95D2F70E945F0C0F900D
:103AF0000F900F900F90CF910C94070CEF92FF92C4
:103B00000F931F93CF93DF938B3109F4EDC008F02F
:103B10008EC08B3009F4B1C008F078C0863009F44B
:103B2000AFC020F4853009F4BDC04EC1873009F420
:103B3000C0C0883009F048C10E9460121F928F9364
:103B400087E199E09F938F930E9486060E945C1202
:103B500083FB992790F91F929F9382FB992790F9F5
:103B60001F929F9381FB992790F91F929F93982F03
:103B700091701F929F931F928F938EEC98E09F936A
:103B80008F930E9486060E94641287FB222720F9E9
:103B90001F922F9386FB222720F91F922F9385FBDC
:103BA000222720F91F922F9384FB222720F91F92AE
:103BB0002F9383FB222720F91F922F9382FB22272A
:103BC00020F91F922F9391FB222720F91F922F9308
:103BD000292F21701F922F9381FB222720F91F92FA
:103BE0002F93282F21701F922F939F938F9389EEED
:103BF00097E09F938F930E9486068DB79EB7889615
:103C00000FB6F8949EBF0FBE8DBF35C0803109F44A
:103C100095C020F48E3009F47BC0D6C0863109F4FB
:103C2000A8C0893109F0D0C08FE595E084C08A3200
:103C3000E1F060F4873209F4C3C028F48E3108F44F
:103C4000C3C08D51BEC0893269F1BEC0833448F40F
:103C50008A3308F0B3C0853309F4B2C0883369F001
:103C6000B3C0833409F4ACC0AFC082EC99E00E94C9
:103C7000ED050E94F912C1E0ACC086E496E05BC09D
:103C800080919802817F8E7F809398028FE196E0E9
:103C90000E94ED058EEB99E00E94ED0581E0809396
:103CA000AE02E9CF82EA99E00E94ED050E94E606A5
:103CB000E2CF80919802C82FC095C170C0FB80F9F7
:103CC00080939802CC2329F086E999E00E94ED05C3
:103CD00080C089E899E00E94ED0580919802897F73
:103CE000877F80939802C7CF9091980291FBCC2751
:103CF000C0F981E0C827892FC0FB81F98093980221
:103D0000CC2319F08CE799E029C08EE699E013C026
:103D10009091980292FBCC27C0F981E0C827892FA7
:103D2000C0FB82F980939802CC2319F08FE599E0CB
:103D300015C08FE499E00E94ED059DCF9091980207
:103D400093FBCC27C0F981E0C827892FC0FB83F9FA
:103D500080939802CC2351F083E499E00E94ED0512
:103D60008091980281608093980233C086E399E045
:103D7000E2CF0E94D021162F072FF82EE92ED091E6
:103D8000CA02C09118010E944C20EF92FF920F933B
:103D90001F931F92DF931F92CF931F928F9384EFF5
:103DA00094E09F938F930E9486068DB79EB70C96E2
:103DB0000FB6F8949EBF0FBE8DBF5DCF895301C073
:103DC00080E00E945E1D57CF84E399E00E94ED05DC
:103DD000C0E08C2FDF91CF911F910F91FF90EF905A
:103DE000089580E008950C94F11ECF93C82F809120
:103DF000AE02813071F040F0823009F045C08C2F66
:103E00000E94411C81E046C00E945A118232F1F5A5
:103E100004C00E945A11823261F48C2F0E94F31E5A
:103E2000811104C08C2F0E947E1D2CC081E090E087
:103E300029C08C2F0E94F11E811123C0C431C9F00A
:103E400058F4CB3069F0C031B9F482E08093AE020F
:103E500088E30E94411C15C0C93259F0C83361F48F
:103E60008FE196E00E94ED058BEE94E00E94ED0557
:103E700008C01092AE020CC089EE94E00E94ED05DD
:103E800007C081E0817006C01092AE0280E002C0DF
:103E900080E0F8CFCF910895CF93DF9386319C4592
:103EA00041F5EB010E945A11982F8A81209102015D
:103EB00030910301882379F09A7A81E009F480E057
:103EC0008093AF02911102C069E201C065E3C901AC
:103ED0000E941D210AC08091AF02811102C069E2D7
:103EE00001C065E3C9010E941F210E949C1180E06E
:103EF00001C081E0DF91CF9108950F931F93CF937D
:103F0000DF93C42FD22FFC0182818823C9F0409314
:103F1000B2020E94C4219093B1028093B00280E269
:103F20008C0F883008F057C0C77081E001C0880F3F
:103F3000CA95EAF7DF91CF911F910F910C94640914
:103F40008091B202481330C08091B0029091B102CA
:103F50000E94DC21883C910538F510E21D0FCD1739
:103F6000B9F080E28C0F883040F4C77081E001C066
:103F7000880FCA95EAF70E946B09183028F581E08E
:103F80009D2F977001C0880F9A95EAF70E946409E7
:103F9000802F0E945B091830F0F4D77081E001C0D7
:103FA000880FDA95EAF70AC080E28C0F883098F41F
:103FB000C77081E001C0880FCA95EAF7DF91CF9101
:103FC0001F910F910C946B09802FDF91CF911F915E
:103FD0000F910C945B09DF91CF911F910F91089580
:103FE0000F939C01CB01243F4CE5340731F188F459
:103FF000293DFCE53F07D9F02A3D4CE5340779F12E
:10400000283D3C45A9F506E221EE41EE68ED7CE550
:104010002BC0263FFCE53F07E1F0A8F0273F3C45D9
:1040200039F507E225EE46EE67EF7CE51DC007E2B5
:1040300025EE45EE69ED7CE517C006E221EE40EE87
:1040400064EF7CE511C007E225EE44EE65EF7CE508
:104050000BC006E221EE42EE66EF7CE505C008E209
:1040600021E045EE6AED7CE50E947D1F80E008C0FE
:10407000FC018281882319F01092B20201C081E014
:104080000F9108959093FD018093FC010895909302
:10409000B8028093B7020895E091B702F091B80298
:1040A000309721F00190F081E02D099480E008958F
:1040B000EF92FF920F931F93CF93DF93E091B7029C
:1040C000F091B8023097B1F18C010280F381E02DBC
:1040D00009958091980282FF2DC080FF04C08BED6E
:1040E00099E00E94ED05E80118E085EDE82E89E0F1
:1040F000F82E8091980280FF0BC088811F928F93C9
:10410000FF92EF920E9486060F900F900F900F90F3
:10411000115021961111EDCF8091980280FF0AC0B5
:1041200083ED99E0DF91CF911F910F91FF90EF9078
:104130000C94ED05DF91CF911F910F91FF90EF90BF
:104140000895E091B702F091B802309739F022E07B
:10415000DC012C930480F581E02D099408952091D1
:10416000B5023091B6022817390771F09093B60264
:104170008093B502E091B702F091B802309721F038
:104180000680F781E02D099408952091B3023091C3
:10419000B4022817390771F09093B4028093B302E8
:1041A000E091B702F091B802309721F00084F185D8
:1041B000E02D09940895FC01329697E080E091503B
:1041C00029F021912223D9F38F5FF9CF0895662337
:1041D00049F0FC01329608962191621729F0E81700
:1041E000F907D1F780E0089581E008959C01FC0172
:1041F00032969FEF80E04191461789F09F3F19F476
:10420000411101C0982F8F5F8630A9F79F3F39F089
:10421000F901E90FF11D97FDFA956283089508955C
:104220009C012A5F3F4FFC014281461301C012826C
:10423000019682179307B9F708950C94F6200C9411
:104240001021029626E0FC0111922A95E9F70895C3
:1042500008950C94282183E08093B9020C942921BD
:10426000811102C081E001C082E08093B9020C9408
:1042700029210C94302181E08093B9020C942921EA
:104280000C943B2108950C9442210C9443210C94EE
:1042900042210C9442210C944221CF930E94492147
:1042A0000E9428170E944721C0E08C2F0E940C1604
:1042B000892B29F4CF5FC530C1F780E001C081E0D0
:1042C000CF91089508951F920F920FB60F92112467
:1042D0008F939F93AF93BF938091BA02811113C0C4
:1042E0008091E1029091E202A091E302B091E40298
:1042F0004196A11DB11D8093E1029093E202A0932B
:10430000E302B093E402BF91AF919F918F910F9020
:104310000FBE0F901F9018958091E902843031F103
:104320000E9466071092BA0220E488E190E00FB67E
:10433000F894A895809360000FBE2093600083B727
:10434000817F846083BF83B7816083BF78948895C1
:1043500083B78E7F83BF0FB6F894A89580916000D5
:10436000886180936000109260000FBE08950E94E3
:10437000070C0C946A0782E084BD93E095BD9AEF28
:1043800097BD80936E0008952FB7F8948091E10255
:104390009091E202A091E302B091E4022FBF089550
:1043A0002FB7F8946091E1027091E2028091E302EC
:1043B0009091E4022FBF08959C014FB7F89480912B
:1043C000E1029091E202A091E302B091E4024FBFBA
:1043D000821B930B089578941F920F920FB60F9241
:1043E00011248F939F93AF93BF938091E10290919B
:1043F000E202A091E302B091E4020196A11DB11D79
:104400008093E1029093E202A093E302B093E4026E
:10441000BF91AF919F918F910F900FBE0F901F9002
:10442000189587E797E790930108809300089AE032
:1044300088E10FB6F894A895809360000FBE909322
:104440006000FFCF8091C9020895089522E0209373
:10445000E9002FEF3091E800215035FD06C035ED21
:104460003A95F1F700002111F5CF2091E80025FFE2
:104470000BC040E050E066E070E00E940E258091A5
:10448000E8008E778093E8000895CF93DF9321E0D2
:104490002093E9002FEF3091E800215035FD06C050
:1044A00035ED3A95F1F700002111F5CF2091E800A4
:1044B00025FF14C0EC0140E050E068E070E00E948D
:1044C0000E258091E8008E778093E80088E0FE0159
:1044D000A1ECB2E001900D928A95E1F7DF91CF91C6
:1044E00008958093BD027093BF026093BE028091D5
:1044F000E902843001F582E08093E9008FEF90912A
:10450000E800815095FD06C095ED9A95F1F7000001
:104510008111F5CF8091E80085FF0DC040E050E0AB
:1045200063E070E08DEB92E00E940E258091E80040
:104530008E778093E8000895BC0184E00C9471228A
:10454000BC0183E00C94712281E09AE00E94ED05A9
:104550008091E802811109C00E949F260E94FC26DA
:104560008091E20084608093E20008958DEF99E0ED
:104570000E94ED051092E802089589EF99E00E94EB
:10458000ED050C94402185EF99E00E94ED056091C6
:10459000E50281E0611101C080E00C942B2181EFE4
:1045A00099E00E94ED059091E90281E0943009F0D4
:1045B00080E06091E5020C9430212091BC022F5FD5
:1045C000822F62E30E94AB29992319F02093BC0249
:1045D00008951092BC028091C002882371F18091ED
:1045E000E902843041F58091E9008F702091EC0060
:1045F000922F917020FD90E8892B93E09093E90031
:104600009091EB0090FF14C09091EE0097FF10C0C6
:104610009091E80095FF03C01092F100F9CF9091BE
:10462000E80090FF05C09091E8009E779093E80025
:104630008F708093E9001092C002089542E061EC0F
:1046400081E00E94182642E261EC82E00E94182676
:1046500042E261EC83E00E9418269091E90281E039
:10466000943009F080E06091E5020C94392180914A
:10467000EB02833009F461C030F4813071F0823094
:1046800009F49AC008958A3009F486C08B3009F481
:104690006CC0893009F0A8C020C08091EA02813A3C
:1046A00009F0A2C08091E800877F8093E8008091A4
:1046B000EE029091EF02892B21F468E081EC92E008
:1046C00003C060E080E090E070E00E945925809196
:1046D000E8008B778093E80008958091EA028132A8
:1046E00009F082C08091EE029091EF02029708F0EB
:1046F0007BC08091E800877F8093E8008091E8008C
:1047000082FD05C08091E9028111F8CF6DC0209132
:10471000F3008091F20090E0922B029731F48091A7
:10472000F100813011F0863021F48091F100809306
:10473000C9028091E8008B7753C08091EA02813AE8
:1047400009F052C08091EE029091EF02892B09F09E
:104750004BC08091E800877F8093E8008091E8005B
:1047600080FFFCCF8091180136C08091EA0281322F
:10477000D9F58091EE029091EF02892BA9F58091F5
:10478000E800877F8093E8000E944D268091EC022C
:10479000809318010C94070C8091EA02813221F574
:1047A0008091E800877F8093E8000E944D268091E9
:1047B000ED028093CA0208958091EA02813AA1F441
:1047C0008091E800877F8093E8008091E80080FF77
:1047D000FCCF8091CA028093F1008091E8008E772F
:1047E0008093E8000C944D2608959FB7F89410929A
:1047F000C0029FBF9091E902943009F057C0909198
:10480000E9009F703091EC00232F217030FD20E8EB
:10481000922B23E02093E9002091EB0020FF43C07E
:104820002091EE0027FF3FC02091BB02222321F000
:104830002091E80025FF37C01092BB0226E030919E
:10484000E80035FD15C03091E902343061F5309152
:10485000EB0035FD28C0215021F481E08093BB029C
:1048600022C0EFE9FFE03197F1F700C00000E7CF89
:104870008093F1008091E80085FD0AC08091E800F6
:1048800080FFFCCF8091E8008E778093E80006C01F
:104890008FB7F89421E02093C0028FBF9F70909350
:1048A000E90080E008959F709093E9008FEF0895EC
:1048B00084B7877F84BF0FB6F894A8958091600075
:1048C000886180936000109260000FBE90E080E8E5
:1048D0000FB6F89480936100909361000FBE0C9422
:1048E0003B210E949F260E94FC26E2EEF0E08081A0
:1048F0008460808378940C9490298CE091E00C94EF
:1049000047208091E9028530C9F48DEE99E00E943C
:10491000ED058091E902853079F40E948C21809127
:10492000E7028823B1F30E944D21882391F30E946E
:10493000F8240E94070CEDCF0C94B7210895089538
:104940000C94A224292F332723303105C9F060F4B9
:104950002130310581F02230310509F041C08BE56D
:1049600090E029E33AE040C021323105E1F0223203
:10497000310531F135C082E190E024E93AE034C0FC
:1049800099278130910549F028F0029749F5E5E033
:10499000FAE005C0E5E3FAE002C0E3E2FAE0849160
:1049A00090E09F0121C063307105D0F4660F771F3E
:1049B000FB01EB50FE4F2081318189E090E014C073
:1049C0006330710568F4FB01EE0FFF1FE151FE4FEC
:1049D00020813181FB01E451FE4F808190E004C0D1
:1049E00080E090E020E030E0FA01318320830895F8
:1049F00080E189BD82E189BD09B400FEFDCF8091CF
:104A0000D8008F7D8093D8008091E00082608093F1
:104A1000E0008091E00081FDFCCF0895CF92DF920D
:104A2000EF92FF920F931F93CF93DF93EC018B01D3
:104A30007A010E946C26811133C0E114F10439F02F
:104A4000F70180819181081B190BC80FD91FC12C58
:104A5000D12C0115110519F18091E80085FD16C0D2
:104A60008091E8008E778093E800E114F10449F02A
:104A7000F70180819181C80ED91ED182C08285E064
:104A80000FC00E946C26882321F30AC0899180936D
:104A9000F10001501109FFEFCF1ADF0ADACF80E0F1
:104AA000DF91CF911F910F91FF90EF90DF90CF900A
:104AB00008952091F0023091F1022617370748F04F
:104AC0006115710539F42091E8002E772093E800F4
:104AD00001C0B901FC0120E06115710579F18091F7
:104AE000E9028823F1F18530F1F18091E80083FD3E
:104AF0003CC08091E80082FD2EC08091E80080FFDC
:104B0000EBCF2091F3008091F20090E0922B6115A1
:104B1000710551F08830910538F421912093F1000E
:104B2000615071090196F3CF21E0089709F020E068
:104B30008091E8008E778093E800CECF2111CFCF0F
:104B40000AC08091E902882361F0853061F080918C
:104B5000E80083FD0AC08091E80082FFF2CF80E088
:104B6000089582E0089583E0089581E008952091FA
:104B7000F0023091F1022617370748F061157105F0
:104B800039F42091E8002E772093E80001C0B901A4
:104B9000FC0120E06115710591F18091E902882303
:104BA00009F440C0853009F43FC08091E80083FDDE
:104BB0003DC08091E80082FD2FC08091E80080FF19
:104BC000E9CF2091F3008091F20090E0922B6115E3
:104BD000710559F08830910540F424912093F1003B
:104BE0003196615071090196F2CF21E0089709F0E2
:104BF00020E08091E8008E778093E800CBCF2111F0
:104C0000CCCF0AC08091E902882361F0853061F041
:104C10008091E80083FD0AC08091E80082FFF2CF16
:104C200080E0089582E0089583E0089581E008958A
:104C3000982F973068F59093E900981739F07091A4
:104C4000EC002091ED005091F00003C0242F762F4E
:104C500050E021FD02C09F5FECCF3091EB003E7F22
:104C60003093EB003091ED003D7F3093ED003091BB
:104C7000EB0031603093EB007093EC002093ED007B
:104C80005093F0002091EE0027FDE5CF80E00895DD
:104C90008F708093E90081E008958091EA0287FF98
:104CA00011C08091E80082FD05C08091E902811168
:104CB000F8CF11C08091E8008B770BC08091E9029A
:104CC000882349F08091E80080FFF8CF8091E800C8
:104CD0008E778093E80008952091E4003091E500FC
:104CE00095E64091EC00842F817040FF23C08091B5
:104CF000E80080FD1DC08091E902882399F085308D
:104D000099F08091EB0085FD11C04091E400509135
:104D1000E5002417350729F3915011F09A01E1CFEE
:104D200084E0089582E0089583E0089581E0089585
:104D300080E008954091E80042FFDDCF08950E9491
:104D40000D270E941527E0EEF0E0808181608083CE
:104D5000E8EDF0E080818F77808319BCA7EDB0E0AB
:104D60008C918E7F8C9380818F7E80831092E8025D
:104D700008950F931F93CF93DF930E940D270E94F6
:104D80001527C8EDD0E088818F7788838881806877
:104D9000888388818F7D888319BC1092E9021092E4
:104DA000E5021092E7021092E60200EE10E0F80130
:104DB00080818B7F808388818160888342E060E08E
:104DC00080E00E941826E1EEF0E080818E7F8083F3
:104DD000E2EEF0E080818160808380818860808362
:104DE000F80180818E7F8083888180618883DF9154
:104DF000CF911F910F910895E8EDF0E080818F7EB3
:104E00008083E7EDF0E080818160808384E082BF71
:104E100081E08093E8020C94B926E8EDF0E080810F
:104E20008E7F80831092E20008951092DA00109233
:104E3000E10008951F920F920FB60F9211242F9345
:104E40003F934F935F936F937F938F939F93AF9312
:104E5000BF93EF93FF938091E10082FF0BC080919D
:104E6000E20082FF07C08091E1008B7F8093E10028
:104E70000E94DD228091DA0080FF1FC08091D8005F
:104E800080FF1BC08091DA008E7F8093DA008091D2
:104E9000D90080FF0DC080E189BD82E189BD09B4E0
:104EA00000FEFDCF81E08093E9020E94A42205C0AC
:104EB00019BC1092E9020E94B6228091E10080FFA5
:104EC00019C08091E20080FF15C08091E2008E7FC2
:104ED0008093E2008091E20080618093E200809103
:104EE000D80080628093D80019BC85E08093E902E5
:104EF0000E94C3228091E10084FF30C08091E200D3
:104F000084FF2CC080E189BD82E189BD09B400FE27
:104F1000FDCF8091D8008F7D8093D8008091E100F3
:104F20008F7E8093E1008091E2008F7E8093E2008B
:104F30008091E20081608093E2008091E502882305
:104F400011F084E007C08091E30087FD02C081E09A
:104F500001C083E08093E9020E94CF228091E100AA
:104F600083FF29C08091E20083FF25C08091E1008A
:104F7000877F8093E10082E08093E9021092E5024E
:104F80008091E1008E7F8093E1008091E2008E7F2E
:104F90008093E2008091E20080618093E20042E031
:104FA00060E080E00E9418268091F0008860809385
:104FB000F0000E94BD22FF91EF91BF91AF919F91B0
:104FC0008F917F916F915F914F913F912F910F90B2
:104FD0000FBE0F901F9018951F920F920FB60F9251
:104FE00011242F933F934F935F936F937F938F93EE
:104FF0009F93AF93BF93CF93DF93EF93FF93C091B2
:10500000E900CF708091EC00D82FD17080FDD0E8FE
:105010001092E9008091F000877F8093F0007894EF
:105020000E9430281092E9008091F00088608093FF
:10503000F000CD2BCF70C093E900FF91EF91DF918D
:10504000CF91BF91AF919F918F917F916F915F9120
:105050004F913F912F910F900FBE0F901F90189579
:105060001F93CF93DF93CDB7DEB7AA970FB6F8940F
:10507000DEBF0FBECDBFEAEEF2E08091F10081937A
:1050800022E0E23FF207C9F70E9437238091E8004F
:1050900083FF2EC18091EA029091EB02492F50E0EC
:1050A0004A30510508F024C1FA01EE59FF4F0C9423
:1050B000CB29803821F0823809F01AC108C08091CC
:1050C000E6029091E702992389F082600FC08091F7
:1050D000EE028F70873008F00BC18093E900809159
:1050E000EB0085FB882780F91092E9009091E80099
:1050F000977F9093E8008093F1001092F100D1C067
:10510000282F2D7F09F0F4C0882319F0823061F038
:10511000EFC08091EC02813009F0EAC0933009F0D1
:1051200080E08093E7022EC08091EC0281112AC0BA
:105130008091EE028F702FEF280F263008F0D8C034
:105140008093E9002091EB0020FF1CC0933021F4F4
:105150008091EB00806214C09091EB00906190937D
:10516000EB0021E030E0A90102C0440F551F8A95F1
:10517000E2F74093EA001092EA008091EB00886029
:105180008093EB001092E9008091E800877F809384
:10519000E8000E944D26ACC08111AAC01091EC021B
:1051A0001F778091E3008078812B8093E3008091CA
:1051B000E800877F8093E8000E944D268091E800F8
:1051C00080FFFCCF8091E30080688093E3001111A1
:1051D00002C082E001C083E08093E90289C0805868
:1051E000823008F085C08091EC029091ED028C3DF8
:1051F00053E0950779F583E08A838AE289834FB784
:10520000F894DE01139620E03EE051E2E32FF0E057
:1052100050935700E49120FF03C0E295EF703F5F89
:10522000EF708E2F90E0EA3010F0C79601C0C09664
:105230008D939D932F5F243149F74FBF8091E800F4
:10524000877F8093E8006AE270E0CE0101960E94B9
:10525000592516C06091EE027091EF02AE014F5FCA
:105260005F4F0E94A024BC01892B09F441C090919A
:10527000E800977F9093E80089819A810E94B72582
:105280008091E8008B778093E80032C0803881F508
:105290008091E800877F8093E8008091E502809309
:1052A000F1008091E8008E7772CF811121C080914A
:1052B000EC029091ED0299270297D4F48091E800D6
:1052C000877F8093E8008091EC028093E5020E9442
:1052D0004D268091E502811106C08091E30087FD93
:1052E00002C081E001C084E08093E9020E941E2395
:1052F0008091E80083FF0AC08091E800877F809357
:10530000E8008091EB0080628093EB00AA960FB6D4
:10531000F894DEBF0FBECDBFDF91CF911F910895EE
:10532000CF938091E9028823A1F0C091E900CF706A
:105330009091EC00892F817090FD80E8C82B10922D
:10534000E9008091E80083FD0E943028CF70C0936F
:10535000E900CF910895991B79E004C0991F961731
:1053600008F0961B881F7A95C9F78095089597FBDA
:10537000072E16F4009407D077FD09D00E94D1299A
:1053800007FC05D03EF4909581959F4F0895709548
:1053900061957F4F0895EE0FFF1F0590F491E02D6A
:1053A0000994AA1BBB1B51E107C0AA1FBB1FA6176C
:1053B000B70710F0A61BB70B881F991F5A95A9F7BE
:1053C00080959095BC01CD010895FB01DC0104C0DE
:1053D0008D910190801921F441505040C8F7881BED
:1053E000990B0895F999FECF92BD81BDF89A99273E
:1053F00080B50895A8E1B0E042E050E00C94262A80
:10540000262FF999FECF92BD81BDF89A019700B47D
:10541000021639F01FBA20BD0FB6F894FA9AF99A1D
:105420000FBE08950396272F0E94012A0E94002A8A
:10543000252F0E94012A242F0C94012A0196272F40
:105440000E94012A0C94002ADC01CB01FC01F9998D
:10545000FECF06C0F2BDE1BDF89A319600B40D92C0
:0C54600041505040B8F70895F894FFCF79
:10546C00C8007C02280850011E0A14012222452281
:10547C002622A0229C22252201E200E900EA00B5A6
:10548C0000B600B700CD008301CC008A01920194D4
:10549C00012102230224022502260227022A02B33A
:1054AC0000B4006F007000818283E200E900EA0022
:1054BC00B500B600B700CD008301CC008A01920183
:1054CC0094012102230224022502260227022A0229
:1054DC00B300B4006F0070008182833230939291DC
:1054EC0090946697C63435363796F0F1F4F5F63F5E
:1054FC003F3F006D6B5F64656C6179006D6B5F693C
:10550C006E74657276616C006D6B5F6D61785F7344
:10551C0070656564006D6B5F74696D655F746F5F5A
:10552C006D6178006D6B5F776865656C5F6D617838
:10553C005F7370656564006D6B5F776865656C5F44
:10554C0074696D655F746F5F6D617800407B224399
:0C555C000BC80AA60A4B0A640A7D0A006C
:00000001FF
